:020000040800F2
:1000000000060020E1020008E3020008E302000805
:10001000E3020008E3020008E3020008E30200082C
:10002000E3020008E3020008E3020008353B000891
:10003000E3020008E3020008E3020008E30200080C
:10004000E3020008E3020008E3020008E3020008FC
:10005000E3020008E3020008193F0008453F0008DA
:10006000713F00089D3F0008C93F0008E3020008F7
:10007000E3020008E3020008E3020008E3020008CC
:10008000E3020008E3020008E3020008E3020008BC
:10009000E3020008E3020008E3020008F53F00085D
:1000A000E3020008E3020008E3020008E30200089C
:1000B000E1400008E3020008E3020008E302000850
:1000C000E3020008E3020008E3020008E30200087C
:1000D000E3020008E3020008E3020008E30200086C
:1000E00059400008E3020008E3020008E3020008A8
:1000F000E3020008E3020008E3020008E30200084C
:10010000E3020008E3020008E3020008E30200083B
:10011000E3020008CD400008E3020008E302000803
:10012000E3020008E3020008E3020008E30200081B
:10013000E3020008E3020008E3020008E30200080B
:10014000E3020008E3020008E3020008E3020008FB
:10015000E3020008E3020008E3020008E3020008EB
:10016000E3020008E3020008E3020008E3020008DB
:10017000E3020008C1340008E3020008E3020008BB
:10018000E3020008E3020008E3020008E3020008BB
:10019000E3020008E3020008E3020008E3020008AB
:1001A000E3020008E3020008E3020008E30200089B
:1001B000E3020008E3020008E3020008E30200088B
:1001C000E3020008E3020008E3020008E30200087B
:1001D000E3020008AD340008E3020008E30200086F
:1001E000E3020008E3020008E3020008E30200085B
:1001F000E3020008E3020008E3020008E30200084B
:10020000E3020008E3020008E3020008E30200083A
:10021000E3020008E3020008E3020008E30200082A
:10022000E3020008E3020008E3020008E30200081A
:10023000E3020008E3020008E3020008E30200080A
:10024000E3020008E3020008E3020008E3020008FA
:10025000E3020008E3020008E3020008E3020008EA
:10026000E3020008E3020008E3020008E3020008DA
:10027000E3020008E3020008E3020008E3020008CA
:10028000E3020008E3020008E3020008E3020008BA
:10029000E3020008E3020008E3020008E3020008AA
:1002A000E3020008E3020008E3020008E30200089A
:1002B000E3020008E3020008E3020008E30200088A
:1002C000E3020008E3020008E3020008E30200087A
:1002D000E3020008E3020008E3020008E30200086A
:1002E00002E000F000F8FEE772B6374880F30888B5
:1002F000364880F3098836483649086040F20000E5
:10030000CCF200004EF63471CEF200010860BFF36B
:100310004F8FBFF36F8F40F20000C0F2F0004EF637
:100320008851CEF200010860BFF34F8FBFF36F8F8B
:100330004FF00000E1EE100A4EF63C71CEF20001E3
:100340000860062080F31488BFF36F8F02F024FB4F
:1003500003F042FB4FF055301F491B4A91423CBF0E
:1003600041F8040BFAE71D49184A91423CBF41F895
:10037000040BFAE71A491B4A1B4B9A423EBF51F83D
:10038000040B42F8040BF8E700201849184A914280
:100390003CBF41F8040BFAE702F03CFB03F0A0FB82
:1003A000144C154DAC4203DA54F8041B8847F9E7A6
:1003B00000F042F8114C124DAC4203DA54F8041B21
:1003C0008847F9E702F024BB000600200022002045
:1003D0000000000808ED00E00000002000060020FA
:1003E0000845000800220020642200206822002026
:1003F000C4470020E0020008E0020008E002000814
:10040000E00200082DE9F04F2DED108AC1F80CD064
:10041000D0F80CD0BDEC108ABDE8F08F002383F338
:1004200011882846A047002001F02CFEFEE701F0CD
:1004300095FD00DFFEE7000038B502F06DFA0546D5
:1004400002F0A0FA0446D0B90F4B9D4219D00133F7
:100450009D4241F2883512BF044600250124002048
:1004600002F064FA0CB100F077F800F071FD00F0D2
:100470001BFC284600F010F900F06EF8F9E70025A3
:10048000EDE70546EBE700BF010007B008B500F057
:10049000D7FBA0F120035842584108BD07B541F2EF
:1004A0001203022101A8ADF8043000F0E7FB03B00D
:1004B0005DF804FB38B5302383F3118817480368CF
:1004C0000BB101F0ABFE0023154A4FF47A711348CB
:1004D00001F09AFE002383F31188124C236813B1B4
:1004E0002368013B2360636813B16368013B636069
:1004F0000D4D2B7833B963687BB9022000F09AFC6C
:10050000322363602B78032B07D163682BB9022059
:1005100000F090FC4FF47A73636038BD68220020CD
:10052000B50400088823002080220020084B1870A2
:1005300003280CD8DFE800F008050208022000F0CC
:1005400069BC022000F058BC024B00225A60704780
:100550008022002088230020F8B5494B494A1C46D8
:100560001968013100F08A8004339342F8D162683F
:10057000454B9A4240F28280444B9B6803F10063F2
:1005800003F500339A4279D2002000F0A7FB022045
:10059000FFF7CCFF3E4B0021D3F8E820C3F8E8106A
:1005A000D3F81021C3F81011D3F81021D3F8EC20A0
:1005B000C3F8EC10D3F81421C3F81411D3F81421A4
:1005C000D3F8F020C3F8F010D3F81821C3F81811AD
:1005D000D3F81821D3F8802042F00072C3F88020AD
:1005E000D3F8802022F00072C3F88020D3F8803046
:1005F00072B64FF0E023C3F8084DD4E90004BFF30E
:100600004F8FBFF36F8F234AC2F88410BFF34F8F11
:10061000536923F480335361BFF34F8FD2F8803096
:1006200043F6E076C3F3C905C3F34E335B0103EA37
:10063000060C29464CEA81770139C2F87472F9D266
:10064000203B13F1200FF2D1BFF34F8FBFF36F8F19
:10065000BFF34F8FBFF36F8F536923F400335361A0
:100660000023C2F85032BFF34F8FBFF36F8F302398
:1006700083F31188854680F308882047F8BD00BFC2
:100680000000020820000208FFFF010800220020ED
:100690000044025800ED00E02DE9F04F93B0B44B58
:1006A0002022FF2100900AA89D6800F0FBFBB14AC0
:1006B0001378A3B90121B04811700360302383F38C
:1006C000118803680BB101F0A9FD0023AB4A4FF478
:1006D0007A71A94801F098FD002383F31188009BEB
:1006E00013B1A74B009A1A60A64A1378032B03D0C4
:1006F00000231370A24A53604FF0000A009CD346B7
:100700005646D146012000F085FB24B19C4B1B6866
:10071000002B00F02682002000F092FA0390039B49
:10072000002BF2DB012000F067FB039B213B1F2B1A
:10073000E8D801A252F823F0B9070008E107000841
:1007400075080008050700080507000805070008E8
:1007500007090008D70A0008F1090008530A000831
:100760007B0A0008A10A000805070008B30A000870
:1007700005070008250B00085908000805070008B0
:10078000690B0008C507000859080008050700089C
:10079000530A0008050700080507000805070008B8
:1007A00005070008050700080507000805070008F9
:1007B00005070008750800080220FFF767FE0028FB
:1007C00040F0F981009B022105A8BAF1000F08BF93
:1007D0001C4641F21233ADF8143000F04FFA91E7A5
:1007E0004FF47A7000F02CFA071EEBDB0220FFF7C3
:1007F0004DFE0028E6D0013F052F00F2DE81DFE844
:1008000007F0030A0D1013360523042105A80593EC
:1008100000F034FA17E004215548F9E704215A485A
:10082000F6E704215948F3E74FF01C08404608F169
:10083000040800F055FA0421059005A800F01EFAFE
:10084000B8F12C0FF2D101204FF0000900FA07F7A0
:1008500047EA0B0B5FFA8BFB00F070FB26B10BF045
:100860000B030B2B08BF0024FFF718FE4AE70421F7
:100870004748CDE7002EA5D00BF00B030B2BA1D1E1
:100880000220FFF703FE074600289BD00120002628
:1008900000F024FA0220FFF749FE5FFA86F840468E
:1008A00000F02CFA0446B0B1039940460136A1F19C
:1008B00040025142514100F031FA0028EDD1BA46D0
:1008C000044641F21213022105A83E46ADF8143049
:1008D00000F0D4F916E725460120FFF727FE244B48
:1008E0009B68AB4207D9284600F0FAF9013040F086
:1008F00067810435F3E70025224BBA463E461D705A
:100900001F4B5D60A8E7002E3FF45CAF0BF00B03BC
:100910000B2B7FF457AF0220FFF708FE322000F0C8
:100920008FF9B0F10008FFF64DAF18F003077FF420
:1009300049AF0F4A08EB0503926893423FF642AF76
:10094000B8F5807F3FF73EAF124BB845019323DDEA
:100950004FF47A7000F074F90390039A002AFFF6BE
:1009600031AF039A0137019B03F8012BEDE700BF7C
:10097000002200208423002068220020B504000803
:10098000882300208022002004220020082200204A
:100990000C22002084220020C820FFF777FD0746A4
:1009A00000283FF40FAF1F2D11D8C5F120020AAB6C
:1009B00025F0030084494245184428BF424601926D
:1009C00000F04AFA019AFF217F4800F06BFA4FEAE3
:1009D000A803C8F387027C492846019300F06AFA0D
:1009E000064600283FF46DAF019B05EB830533E716
:1009F0000220FFF74BFD00283FF4E4AE00F0ACF915
:100A000000283FF4DFAE0027B846704B9B68BB421E
:100A100018D91F2F11D80A9B01330ED027F00303DA
:100A200012AA134453F8203C05934046042205A91A
:100A3000043700F0F1FA8046E7E7384600F050F955
:100A40000590F2E7CDF81480042105A800F016F90E
:100A500002E70023642104A8049300F005F90028AC
:100A60007FF4B0AE0220FFF711FD00283FF4AAAEDC
:100A7000049800F067F90590E6E70023642104A8D4
:100A8000049300F0F1F800287FF49CAE0220FFF7F9
:100A9000FDFC00283FF496AE049800F055F9EAE713
:100AA0000220FFF7F3FC00283FF48CAE00F064F95D
:100AB000E1E70220FFF7EAFC00283FF483AE05A936
:100AC000142000F05FF907460421049004A800F008
:100AD000D5F83946B9E7322000F0B2F8071EFFF624
:100AE00071AEBB077FF46EAE384A07EB090392681C
:100AF00093423FF667AE0220FFF7C8FC00283FF4A0
:100B000061AE27F003074F44B9453FF4A5AE484610
:100B100009F1040900F0E4F80421059005A800F0AB
:100B2000ADF8F1E74FF47A70FFF7B0FC00283FF41E
:100B300049AE00F011F9002844D00A9B01330BD0D4
:100B400008220AA9002000F0B5F900283AD0202296
:100B5000FF210AA800F0A6F9FFF7A0FC1C4801F04D
:100B600097FA13B0BDE8F08F002E3FF42BAE0BF0D8
:100B70000B030B2B7FF426AE0023642105A80593FD
:100B800000F072F8074600287FF41CAE0220FFF741
:100B90007DFC804600283FF415AEFFF77FFC41F254
:100BA000883001F075FA059800F014FA46463C4684
:100BB00000F0C4F9A6E506464EE64FF0000901E64E
:100BC000BA467EE637467CE68422002000220020DA
:100BD000A08601002DE9F84F4FF47A7306460D46C2
:100BE000002402FB03F7DFF85080DFF8509098F9FB
:100BF00000305FFA84FA5A1C01D0A34212D159F88E
:100C000024002A4631460368D3F820B03B46D84733
:100C1000854207D1074B012083F800A0BDE8F88F7B
:100C20000124E4E7002CFBD04FF4FA7001F030FA15
:100C30000020F3E7D42300201022002014220020FB
:100C4000002307B5024601210DF107008DF807309A
:100C5000FFF7C0FF20B19DF8070003B05DF804FB6B
:100C60004FF0FF30F9E700000A46042108B5FFF70E
:100C7000B1FF80F00100C0B2404208BD074B0A46F8
:100C800030B41978064B53F82140014623682046BA
:100C9000DD69044BAC4630BC604700BFD423002064
:100CA00014220020A086010070B50A4E00240A4DCF
:100CB00001F00AFD308028683388834208D901F0AA
:100CC000FFFC2B6804440133B4F5003F2B60F2D3E2
:100CD00070BD00BFD62300209023002001F0D2BDBC
:100CE00000F1006000F500300068704700F100601E
:100CF000920000F5003001F049BD0000054B1A6874
:100D0000054B1B889B1A834202D9104401F0D8BCC2
:100D10000020704790230020D623002038B50446D9
:100D2000074D29B128682044BDE8384001F0E0BCF7
:100D30002868204401F0CAFC0028F3D038BD00BF69
:100D4000902300200020704700F1FF5000F58F1025
:100D5000D0F8000870470000064991F8243033B1FC
:100D600000230822086A81F82430FFF7BFBF012062
:100D7000704700BF94230020014B1868704700BFE4
:100D80000010005C194B01380322084470B51D683F
:100D9000174BC5F30B042D0C1E88A6420BD15C68C3
:100DA0000A46013C824213460FD214F9016F4EB13C
:100DB00002F8016BF6E7013A03F10803ECD1814236
:100DC0000B4602D22C2203F8012B0424094A168870
:100DD000AE4204D1984284BF967803F8016B013C7F
:100DE00002F10402F3D1581A70BD00BF0010005C7C
:100DF0001C220020E4410008022803D1044B0822F1
:100E00009A6170470128FCD1014B0422F8E700BF2A
:100E100000100258022804D1054B4FF400229A61B9
:100E200070470128FCD1024B4FF48022F7E700BF46
:100E300000100258022805D1064A536983F00803BE
:100E4000536170470128FCD1024A536983F00403BF
:100E5000F6E700BF00100258002310B5934203D0FC
:100E6000CC5CC4540133F9E710BD0000013810B563
:100E700010F9013F3BB191F900409C4203D11AB1F6
:100E80000131013AF4E71AB191F90020981A10BD26
:100E90001046FCE703460246D01A12F9011B00294E
:100EA000FAD1704702440346934202D003F8011B73
:100EB000FAE770472DE9F8431F4D14460746884668
:100EC00095F8242052BBDFF870909CB395F824303D
:100ED0002BB92022FF2148462F62FFF7E3FF95F848
:100EE00024004146C0F1080205EB8000A24228BF61
:100EF0002246D6B29200FFF7AFFF95F82430A41B2C
:100F000017441E449044E4B2F6B2082E85F82460DB
:100F1000DBD1FFF721FF0028D7D108E02B6A03EBD4
:100F200082038342CFD0FFF717FF0028CBD10020E8
:100F3000BDE8F8830120FBE794230020024B1A78D8
:100F4000024B1A70704700BFD423002010220020EB
:100F500038B51A4C1A4D204600F0C8FB29462046E9
:100F600000F0F0FB2D681748D5F89020D2F804382F
:100F700043F00203C2F8043801F08AF81249284607
:100F800000F0EEFCD5F89020104DD2F80438286817
:100F900023F002030E49A042C2F804384FF4E133B3
:100FA0000B6001D000F000FB6868A04204D0084943
:100FB000BDE8384000F0F8BA38BD00BFB82A0020BC
:100FC000E042000840420F00E842000814220020DE
:100FD000BC2300200C4B70B50C4D04461E780C4B06
:100FE00055F826209A420DD00A4B002118221846A7
:100FF000FFF758FF0460014655F82600BDE8704031
:1010000000F0D2BA70BD00BFD4230020142200200B
:10101000B82A0020BC23002030B50A44084D914274
:101020000DD011F8013B5840082340F30004013B68
:101030002C4013F0FF0384EA5000F6D1EFE730BDF7
:101040002083B8ED026843681143016003B118477B
:1010500070470000024A136843F0C00313607047F2
:101060000050004013B50E4C204600F091FA04F1F8
:10107000140000234FF400720A49009400F04EF966
:10108000094B4FF40072094904F13800009400F054
:10109000C7F9074A074BC4E9172302B010BD00BFC8
:1010A000D8230020442400205510000844260020A6
:1010B0000050004000E1F505037C30B5244C0029C8
:1010C00018BF0C46012B11D1224B98420ED1224B56
:1010D000D3F8E82042F48012C3F8E820D3F81021B6
:1010E00042F48012C3F81021D3F810312268036E45
:1010F000C16D03EB52038466B3FBF2F3626815041F
:1011000042BF23F0070503F0070343EA4503CB6022
:10111000A36843F040034B60E36843F001038B6036
:1011200042F4967343F001030B604FF0FF330B6200
:10113000510505D512F0102205D0B2F1805F04D020
:1011400080F8643030BD7F23FAE73F23F8E700BF23
:10115000F4410008D8230020004402582DE9F0474C
:10116000C66D05463768F469210734621AD014F059
:10117000080118BF4FF48071E20748BF41F0200119
:10118000A3074FF0300348BF41F04001600748BF5C
:1011900041F0800183F31188281DFFF753FF0023DE
:1011A00083F31188E2050AD5302383F311884FF4C5
:1011B0008061281DFFF746FF002383F311884FF05D
:1011C00030094FF0000A14F0200838D13B0616D53C
:1011D0004FF0300905F1380A200610D589F311883F
:1011E000504600F051F9002836DA0821281DFFF793
:1011F00029FF27F080033360002383F311887906E9
:1012000014D5620612D5302383F31188D5E9132350
:101210009A4208D12B6C33B127F040071021281DCA
:10122000FFF710FF3760002383F31188E30618D51A
:10123000AA6E1369ABB15069BDE8F047184789F34E
:101240001188736A284695F86410194000F0BAF9BD
:101250008AF31188F469B6E7B06288F31188F469FB
:10126000BAE7BDE8F0870000F8B515468268044685
:101270000B46AA4200D28568A1692669761AB54252
:101280000BD218462A46FFF7E7FDA3692B44A3615A
:101290002846A3685B1BA360F8BD0CD9AF1B18469A
:1012A0003246FFF7D9FD3A46E1683044FFF7D4FDF6
:1012B000E3683B44EBE718462A46FFF7CDFDE368B9
:1012C000E5E7000083689342F7B50446154600D26F
:1012D0008568D4E90460361AB5420BD22A46FFF776
:1012E000BBFD63692B4463612846A3685B1BA36055
:1012F00003B0F0BD0DD93246AF1B0191FFF7ACFD35
:1013000001993A46E0683144FFF7A6FDE3683B44A3
:10131000E9E72A46FFF7A0FDE368E4E710B50A44D1
:101320000024C361029B8460C16002610362C0E962
:101330000000C0E9051110BD08B5D0E9053293429F
:1013400001D1826882B98268013282605A1C42618E
:1013500019700021D0E904329A4224BFC368436166
:1013600000F0B2FE002008BD4FF0FF30FBE70000A8
:1013700070B5302304460E4683F31188A568A5B1E5
:10138000A368A269013BA360531CA361157822697D
:10139000934224BFE368A361E3690BB120469847F9
:1013A000002383F31188284607E03146204600F0E9
:1013B0007BFE0028E2DA85F3118870BD2DE9F74F36
:1013C00004460E4617469846D0F81C904FF0300A57
:1013D0008AF311884FF0000B154665B12A46314655
:1013E0002046FFF741FF034660B94146204600F022
:1013F0005BFE0028F1D0002383F31188781B03B033
:10140000BDE8F08FB9F1000F03D001902046C84726
:10141000019B8BF31188ED1A1E448AF31188DCE7D7
:10142000C160C361009B82600362C0E90511114481
:10143000C0E9000001617047F8B504460D46164644
:10144000302383F31188A768A7B1A368013BA36089
:1014500063695A1C62611D70D4E904329A4224BF48
:10146000E3686361E3690BB120469847002080F38D
:10147000118807E03146204600F016FE0028E2DA27
:1014800087F31188F8BD0000D0E9052310B59A4212
:1014900001D182687AB982680021013282605A1CC7
:1014A00082611C7803699A4224BFC368836100F09B
:1014B0000BFE204610BD4FF0FF30FBE72DE9F74F44
:1014C00004460E4617469846D0F81C904FF0300A56
:1014D0008AF311884FF0000B154665B12A46314654
:1014E0002046FFF7EFFE034660B94146204600F074
:1014F000DBFD0028F1D0002383F31188781B03B0B3
:10150000BDE8F08FB9F1000F03D001902046C84725
:10151000019B8BF31188ED1A1E448AF31188DCE7D6
:10152000026843681143016003B118477047000027
:101530001430FFF743BF00004FF0FF331430FFF7C4
:101540003DBF00003830FFF7B9BF00004FF0FF3358
:101550003830FFF7B3BF00001430FFF709BF0000B9
:101560004FF0FF311430FFF703BF00003830FFF7B2
:1015700063BF00004FF0FF323830FFF75DBF00005F
:10158000012914BF6FF0130000207047FFF76ABDF8
:10159000044B036000234360C0E90233012303745A
:1015A000704700BF0C42000810B53023044683F397
:1015B0001188FFF781FD02230020237480F3118836
:1015C00010BD000038B5C36904460D461BB904219F
:1015D0000844FFF7A5FF294604F11400FFF7ACFE0D
:1015E000002806DA201D4FF40061BDE83840FFF7FF
:1015F00097BF38BD026843681143016003B11847C3
:101600007047000013B5406B00F58054D4F8A4383F
:101610001A681178042914D1017C022911D1197991
:10162000012312898B4013420BD101A94C3002F0E7
:101630008FF8D4F8A4480246019B2179206800F075
:10164000DFF902B010BD0000143002F011B8000044
:101650004FF0FF33143002F00BB800004C3002F0B2
:10166000E3B800004FF0FF334C3002F0DDB800006B
:10167000143001F0DFBF00004FF0FF31143001F0F3
:10168000D9BF00004C3002F0AFB800004FF0FF327D
:101690004C3002F0A9B800000020704710B500F5EA
:1016A0008054D4F8A4381A681178042917D1017C21
:1016B000022914D15979012352898B4013420ED14A
:1016C000143001F071FF024648B1D4F8A4484FF439
:1016D000407361792068BDE8104000F07FB910BD0B
:1016E000406BFFF7DBBF0000704700007FB5124B77
:1016F00001250426044603600023057400F18402DA
:1017000043602946C0E902330C4B02901430019328
:101710004FF44073009601F023FF094B04F6944206
:10172000294604F14C000294CDE900634FF4407364
:1017300001F0EAFF04B070BD34420008E116000871
:10174000051600080A68302383F311880B790B33E0
:1017500042F823004B79133342F823008B7913B1FD
:101760000B3342F8230000F58053C3F8A41802237A
:101770000374002080F311887047000038B5037FA0
:10178000044613B190F85430ABB90125201D022155
:10179000FFF730FF04F114006FF00101257700F02E
:1017A0009FFC04F14C0084F854506FF00101BDE837
:1017B000384000F095BC38BD10B501210446043016
:1017C000FFF718FF0023237784F8543010BD000082
:1017D00038B504460025143001F0DAFE04F14C005F
:1017E000257701F0A9FF201D84F854500121FFF74F
:1017F00001FF2046BDE83840FFF750BF90F8803029
:1018000003F06003202B06D190F881200023212AC9
:1018100003D81F2A06D800207047222AFBD1C0E92E
:101820001D3303E0034A426707228267C367012032
:10183000704700BF3422002037B500F58055D5F839
:10184000A4381A68117804291AD1017C022917D109
:101850001979012312898B40134211D100F14C04F4
:10186000204602F029F858B101A9204601F070FF86
:10187000D5F8A4480246019B2179206800F0C0F801
:1018800003B030BD01F10B03F0B550F8236085B013
:1018900004460D46FEB1302383F3118804EB85071F
:1018A000301D0821FFF7A6FEFB6806F14C005B69BE
:1018B0001B681BB1019001F059FF019803A901F0C9
:1018C00047FF024648B1039B2946204600F098F89E
:1018D000002383F3118805B0F0BDFB685A691268D4
:1018E000002AF5D01B8A013B1340F1D104F180029C
:1018F000EAE70000133138B550F82140ECB130234D
:1019000083F3118804F58053D3F8A428136852791F
:1019100003EB8203DB689B695D6845B104216018B5
:10192000FFF768FE294604F1140001F047FE204647
:10193000FFF7B4FE002383F3118838BD7047000021
:1019400001F0FEB801234022002110B5044600F842
:10195000303BFFF7A7FA0023C4E9013310BD0000B4
:1019600010B53023044683F31188242241600021FE
:101970000C30FFF797FA204601F004F9022300200B
:10198000237080F3118810BD70B500EB810305460C
:1019900050690E461446DA6018B110220021FFF794
:1019A00081FAA06918B110220021FFF77BFA3146B5
:1019B0002846BDE8704001F0EBB9000083682022A2
:1019C000002103F0011310B5044683601030FFF7C7
:1019D00069FA2046BDE8104001F066BAF0B401256E
:1019E00000EB810447898D40E4683D43A46945814B
:1019F00023600023A2606360F0BC01F083BA0000A2
:101A0000F0B4012500EB810407898D40E4683D4373
:101A10006469058123600023A2606360F0BC01F06B
:101A2000F9BA000070B50223002504462422037091
:101A30002946C0F888500C3040F8045CFFF732FAB1
:101A4000204684F8705001F037F963681B6823B1B1
:101A500029462046BDE87040184770BD0378052B25
:101A600010B504460AD080F88C3005230370436813
:101A70001B680BB1042198470023A36010BD000030
:101A80000178052906D190F88C20436802701B6804
:101A900003B118477047000070B590F870300446E5
:101AA00013B1002380F8703004F18002204601F069
:101AB0001FFA63689B68B3B994F8803013F060052F
:101AC00035D00021204601F011FD0021204601F013
:101AD00001FD63681B6813B1062120469847062361
:101AE00084F8703070BD204698470028E4D0B4F8E0
:101AF0008630A26F9A4288BFA36794F98030A56FA1
:101B0000002B4FF0300380F20381002D00F0F280B3
:101B1000092284F8702083F3118800212046D4E93B
:101B20001D23FFF76DFF002383F31188DAE794F894
:101B3000812003F07F0343EA022340F20232934202
:101B400000F0C58021D8B3F5807F48D00DD8012B97
:101B50003FD0022B00F09380002BB2D104F1880219
:101B600062670222A267E367C1E7B3F5817F00F0F5
:101B70009B80B3F5407FA4D194F88230012BA0D193
:101B8000B4F8883043F0020332E0B3F5006F4DD073
:101B900017D8B3F5A06F31D0A3F5C063012B90D84F
:101BA0006368204694F882205E6894F88310B4F845
:101BB0008430B047002884D0436863670368A36714
:101BC0001AE0B3F5106F36D040F6024293427FF42C
:101BD00078AF5C4B63670223A3670023C3E794F8E5
:101BE0008230012B7FF46DAFB4F8883023F002030C
:101BF000A4F88830C4E91D55E56778E7B4F880306B
:101C0000B3F5A06F0ED194F88230204684F88A3064
:101C100001F0B0F863681B6813B1012120469847B2
:101C2000032323700023C4E91D339CE704F18B03D5
:101C300063670123C3E72378042B10D1302383F398
:101C400011882046FFF7BAFE85F3118803216368E7
:101C500084F88B5021701B680BB12046984794F88C
:101C60008230002BDED084F88B300423237063682D
:101C70001B68002BD6D0022120469847D2E794F863
:101C8000843020461D0603F00F010AD501F022F929
:101C9000012804D002287FF414AF2B4B9AE72B4B7A
:101CA00098E701F009F9F3E794F88230002B7FF40C
:101CB00008AF94F8843013F00F01B3D01A06204611
:101CC00002D501F02BFCADE701F01CFCAAE794F86B
:101CD0008230002B7FF4F5AE94F8843013F00F01BE
:101CE000A0D01B06204602D501F000FC9AE701F0C7
:101CF000F1FB97E7142284F8702083F311882B46B8
:101D00002A4629462046FFF769FE85F31188E9E651
:101D10005DB1152284F8702083F3118800212046DC
:101D2000D4E91D23FFF75AFEFDE60B2284F870204C
:101D300083F311882B462A4629462046FFF760FE8A
:101D4000E3E700BF644200085C420008604200080C
:101D500038B590F870300446002B3ED0063BDAB21E
:101D60000F2A34D80F2B32D8DFE803F0373131088F
:101D7000223231313131313131313737856FB0F87D
:101D800086309D4214D2C3681B8AB5FBF3F203FB75
:101D900012556DB9302383F311882B462A46294604
:101DA000FFF72EFE85F311880A2384F870300EE0C9
:101DB000142384F87030302383F3118800232046E5
:101DC0001A461946FFF70AFE002383F3118838BD2F
:101DD000C36F03B198470023E7E70021204601F0D5
:101DE00085FB0021204601F075FB63681B6813B179
:101DF0000621204698470623D7E7000010B590F843
:101E000070300446142B29D017D8062B05D001D8E2
:101E10001BB110BD093B022BFBD80021204601F06D
:101E200065FB0021204601F055FB63681B6813B178
:101E3000062120469847062319E0152BE9D10B23EC
:101E400080F87030302383F3118800231A46194636
:101E5000FFF7D6FD002383F31188DAE7C3689B6997
:101E60005B68002BD5D1C36F03B19847002384F87A
:101E70007030CEE700238268037503691B68996898
:101E80009142FBD25A68036042601060586070470C
:101E900000238268037503691B6899689142FBD827
:101EA0005A680360426010605860704708B5084681
:101EB000302383F311880B7D032B05D0042B0DD029
:101EC0002BB983F3118808BD8B6900221A604FF08B
:101ED000FF338361FFF7CEFF0023F2E7D1E9003241
:101EE00013605A60F3E70000FFF7C4BF054BD968E1
:101EF00008751868026853601A600122D86002757C
:101F0000FEF780BA482800200C4B30B5DD684B1C2A
:101F100087B004460FD02B46094A684600F074F992
:101F20002046FFF7E3FF009B13B1684600F076F907
:101F3000A86907B030BDFFF7D9FFF9E748280020AE
:101F4000AD1E0008044B1A68DB6890689B689842D5
:101F500094BF00200120704748280020084B10B58E
:101F60001C68D868226853601A600122DC60227500
:101F7000FFF78EFF01462046BDE81040FEF742BA4B
:101F800048280020044B1A68DB6892689B689A42D4
:101F900001D9FFF7E3BF70474828002038B5074C48
:101FA00001230025064907482370656001F0BCFC49
:101FB0000223237085F3118838BD00BFB02A0020AA
:101FC0006C4200084828002000F05EB9EFF3118051
:101FD00020B9EFF30583302282F3118870470000A7
:101FE00010B530B9EFF30584C4F3080414B180F3DD
:101FF000118810BDFFF7C6FF84F31188F9E70000D0
:10200000034A516853685B1A9842FBD8704700BF77
:10201000001000E08B600223086108468B82704745
:102020008368A3F1840243F8142C026943F8442C1A
:10203000426943F8402C094A43F8242CC268A3F1B2
:10204000200043F8182C022203F80C2C002203F87D
:102050000B2C034A43F8102C704700BF1D040008E6
:102060004828002008B5FFF7DBFFBDE80840FFF770
:102070003BBF0000024BDB6898610F20FFF736BFC3
:1020800048280020302383F31188FFF7F3BF0000B6
:1020900008B50146302383F311880820FFF734FF89
:1020A000002383F3118808BD064BDB6839B1426811
:1020B00018605A60136043600420FFF725BF4FF09B
:1020C000FF307047482800200368984206D01A68FD
:1020D0000260506018469961FFF706BF7047000024
:1020E00038B504460D462068844200D138BD0368E7
:1020F00023605C608561FFF7F7FEF4E7036810B5C5
:102100009C68A2420CD85C688A600B604C602160BD
:10211000596099688A1A9A604FF0FF33836010BD46
:10212000121B1B68ECE700000A2938BF0A2170B5B2
:1021300004460D460A26601901F0F0FB01F0DCFBB5
:10214000041BA54203D8751C04462E46F3E70A2E4D
:1021500004D90120BDE8704001F026BC70BD00002C
:10216000F8B5144B0D460A2A4FF00A07D96103F15E
:102170001001826038BF0A2241601969144601606B
:1021800048601861A81801F0BBFB01F0B5FB431BC8
:102190000646A34206D37C1C28192746354601F083
:1021A000BDFBF2E70A2F04D90120BDE8F84001F099
:1021B000FBBBF8BD48280020F8B506460D4601F0E7
:1021C0009BFB0F4A134653F8107F9F4206D12A46C5
:1021D00001463046BDE8F840FFF7C2BFD169BB6891
:1021E000441A2C1928BF2C46A34202D92946FFF7CE
:1021F0009BFF224631460348BDE8F840FFF77EBF0B
:102200004828002058280020C0E90323002310B4E8
:102210005DF8044B4361FFF7CFBF000010B5194CC8
:10222000236998420DD08168D0E9003213605A606A
:102230009A680A449A60002303604FF0FF33A36159
:1022400010BD0268234643F8102F5360002202603D
:1022500022699A4203D1BDE8104001F059BB93684E
:1022600081680B44936001F047FB2269E169926841
:10227000441AA242E4D91144BDE81040091AFFF7FC
:1022800053BF00BF482800202DE9F047DFF8BC808D
:1022900008F110072C4ED8F8105001F02DFBD8F89B
:1022A0001C40AA68031B9A423ED814444FF0000910
:1022B000D5E90032C8F81C4013605A60C5F8009098
:1022C000D8F81030B34201D101F022FB89F3118814
:1022D000D5E9033128469847302383F311886B6989
:1022E000002BD8D001F008FB6A69A0EB04098246F4
:1022F0004A450DD2022001F057FB0022D8F81030D9
:10230000B34208D151462846BDE8F047FFF728BF41
:10231000121A2244F2E712EB09092946384638BF5F
:102320004A46FFF7EBFEB5E7D8F81030B34208D0C5
:102330001444C8F81C00211AA960BDE8F047FFF753
:10234000F3BEBDE8F08700BF5828002048280020D1
:1023500000207047FEE70000704700004FF0FF309C
:102360007047000002290CD0032904D00129074836
:1023700018BF00207047032A05D8054800EBC200AB
:102380007047044870470020704700BF444300086E
:1023900044220020F842000870B59AB0054608466D
:1023A000144601A900F0C2F801A8FEF773FD431C12
:1023B0000022C6B25B001046C5E900342370032337
:1023C000023404F8013C01ABD1B202348E4201D890
:1023D0001AB070BD13F8011B013204F8010C04F8A7
:1023E000021CF1E708B5302383F311880348FFF797
:1023F00023FA002383F3118808BD00BFB82A002008
:1024000090F8803003F01F02012A07D190F8812054
:102410000B2A03D10023C0E91D3315E003F060034C
:10242000202B08D1B0F884302BB990F88120212AD4
:1024300003D81F2A04D8FFF7E1B9222AEBD0FAE724
:10244000034A426707228267C3670120704700BFC3
:102450003B22002007B5052917D8DFE801F019163F
:1024600003191920302383F31188104A01210190A8
:10247000FFF78AFA019802210D4AFFF785FA0D4805
:10248000FFF7A6F9002383F3118803B05DF804FB7E
:10249000302383F311880748FFF770F9F2E7302300
:1024A00083F311880348FFF787F9EBE798420008A8
:1024B000BC420008B82A002038B50C4D0C4C2A4606
:1024C0000C4904F10800FFF767FF05F1CA0204F1A7
:1024D00010000949FFF760FF05F5CA7204F1180002
:1024E0000649BDE83840FFF757BF00BF90430020C2
:1024F0004422002078420008824200088D420008F1
:1025000070B5044608460D46FEF7C4FCC6B2204628
:10251000013403780BB9184670BD32462946FEF7E0
:10252000A5FC0028F3D10120F6E700002DE9F047D3
:1025300005460C46FEF7AEFC2B49C6B22846FFF70F
:10254000DFFF08B10736F6B228492846FFF7D8FF63
:1025500008B11036F6B2632E0BD8DFF88C80DFF8A6
:102560008C90234FDFF894A02E7846B92670BDE8F2
:10257000F08729462046BDE8F04701F015BE252E1C
:102580002ED1072241462846FEF770FC70B9194B40
:10259000224603F10C0153F8040B8B4242F8040B62
:1025A000F9D11B8807350E341380DDE70822494630
:1025B0002846FEF75BFC98B9A21C0F4B1978023233
:1025C0000909C95D02F8041C13F8011B01F00F0191
:1025D0005345C95D02F8031CF0D118340835C3E730
:1025E000013504F8016BBFE7644300088D42000821
:1025F0007B4300086C43000800E8F11F0CE8F11F62
:10260000BFF34F8F044B1A695107FCD1D3F8102147
:102610005207F8D1704700BF0020005208B50D4B9B
:102620001B78ABB9FFF7ECFF0B4BDA68D10704D589
:102630000A4A5A6002F188325A60D3F80C21D20754
:1026400006D5064AC3F8042102F18832C3F80421F2
:1026500008BD00BFEE450020002000522301674561
:1026600008B5114B1B78F3B9104B1A69510703D504
:10267000DA6842F04002DA60D3F81021520705D53B
:10268000D3F80C2142F04002C3F80C21FFF7B8FF49
:10269000064BDA6842F00102DA60D3F80C2142F00E
:1026A0000102C3F80C2108BDEE45002000200052B5
:1026B0000F289ABF00F5806040040020704700009A
:1026C0004FF4003070470000102070470F2808B505
:1026D0000BD8FFF7EDFF00F500330268013204D19B
:1026E00004308342F9D1012008BD0020FCE700003E
:1026F0000F2870B5054645D8FFF768FC224CFFF758
:102700007FFF0646FFF78AFF4FF0FF33072D636117
:10271000C4F8143120D82361FFF772FF2B0243F075
:102720002403E360E36843F08003E36023695A070E
:10273000FCD42846FFF764FF4FF40031FFF7B8FFE1
:1027400000F002F93046FFF78BFFFFF749FC2846FF
:10275000BDE87040FFF7BABFC4F81031FFF750FF73
:10276000A5F108031B0243F02403C4F80C31D4F88C
:102770000C3143F08003C4F80C31D4F810315B07FE
:10278000FBD4D6E7002070BD002000522DE9F84FA1
:1027900040EA020305460C461746D80602D0002040
:1027A000BDE8F88F27F01F07DFF8D4B0FFF736FF3A
:1027B0002744BC4203D10120FFF752FFF0E720225B
:1027C0002946204601F0E0FC10B920352034F0E71E
:1027D0002B4605F120021E68711CE0D104339A4299
:1027E000F9D1FFF7F3FB05F17843234AB3F5801FD6
:1027F000224B28BF9A4603F1040338BF9046A2F14A
:10280000080228BF9846A3F108033ABF9146DA466A
:102810009946FFF7F5FEC8F80060A5EB040CD9F85F
:10282000002004F11C0142F00202C9F80020221F1E
:10283000DAF8006016F00506FAD152F8043F8A4231
:102840004CF80230F4D1BFF34F8FFFF7D9FE4FF0B1
:10285000FF32C8F80020D9F8002022F00202C9F89F
:102860000020FFF7BDFB20222146284601F08CFC0A
:102870000028AAD030469FE71420005210210052B1
:102880001020005210B5084C237828B11BB9FFF76F
:10289000C5FE0123237010BD002BFCD02070BDE8C5
:1028A0001040FFF7DDBE00BFEE4500200244074B9D
:1028B000D2B210B5904200D110BD441C00B253F802
:1028C000200041F8040BE0B2F4E700BF504000588C
:1028D0000E4B30B51C6F240405D41C6F1C671C6F95
:1028E00044F400441C670A4C02442368D2B243F407
:1028F00080732360074B904200D130BD441C51F8D7
:10290000045B00B243F82050E0B2F4E70044025800
:10291000004802585040005807B5012201A9002084
:10292000FFF7C4FF019803B05DF804FB13B504463C
:10293000FFF7F2FFA04205D0012201A90020019477
:10294000FFF7C6FF02B010BD0144BFF34F8F064B27
:10295000884204D3BFF34F8FBFF36F8F7047C3F824
:102960005C022030F4E700BF00ED00E0034B1A6882
:102970001AB9034AD2F8D0241A607047F0450020F3
:102980000040025808B5FFF7F1FF024B1868C0F38A
:10299000806008BDF045002070B5BFF34F8FBFF3D6
:1029A0006F8F1A4A0021C2F85012BFF34F8FBFF346
:1029B0006F8F536943F400335361BFF34F8FBFF3FD
:1029C0006F8FC2F88410BFF34F8FD2F8803043F678
:1029D000E074C3F3C900C3F34E335B0103EA04069A
:1029E000014646EA81750139C2F86052F9D2203BAE
:1029F00013F1200FF2D1BFF34F8F536943F48033AB
:102A00005361BFF34F8FBFF36F8F70BD00ED00E0D8
:102A1000FEE70000214B2248224A70B5904237D38E
:102A2000214BC11EDA1C121A22F003028B4238BF5E
:102A300000220021FEF736FA1C4A0023C2F8843037
:102A4000BFF34F8FD2F8803043F6E074C3F3C90070
:102A5000C3F34E335B0103EA0406014646EA81757F
:102A60000139C2F86C52F9D2203B13F1200FF2D198
:102A7000BFF34F8FBFF36F8FBFF34F8FBFF36F8FD6
:102A80000023C2F85032BFF34F8FBFF36F8F70BD7A
:102A900053F8041B40F8041BC0E700BF6C45000856
:102AA000C4470020C4470020C447002000ED00E0D8
:102AB000074BD3F8D81021EA0001C3F8D810D3F897
:102AC000002122EA0002C3F80021D3F80031704748
:102AD0000044025870B5D0E9244300224FF0FF357E
:102AE0009E6804EB42135101D3F80009002805DA6F
:102AF000D3F8000940F08040C3F80009D3F8000B78
:102B0000002805DAD3F8000B40F08040C3F8000B32
:102B1000013263189642C3F80859C3F8085BE0D243
:102B20004FF00113C4F81C3870BD0000890141F05A
:102B30002001016103699B06FCD41220FFF760BAF3
:102B400010B50A4C2046FEF7FDFE094BC4F8903044
:102B5000084BC4F89430084C2046FEF7F3FE074BB0
:102B6000C4F89030064BC4F8943010BDF4450020F2
:102B700000000840B04300089046002000000440D8
:102B8000BC43000870B503780546012B5CD1434B6C
:102B9000D0F89040984258D1414B0E216520D3F88F
:102BA000D82042F00062C3F8D820D3F8002142F0C8
:102BB0000062C3F80021D3F80021D3F8802042F04E
:102BC0000062C3F88020D3F8802022F00062C3F8AE
:102BD0008020D3F8803000F0ADFC324BE360324B04
:102BE000C4F800380023D5F89060C4F8003EC02334
:102BF00023604FF40413A3633369002BFCDA012331
:102C00000C203361FFF7FCF93369DB07FCD4122099
:102C1000FFF7F6F93369002BFCDA00262846A66098
:102C2000FFF758FF6B68C4F81068DB68C4F81468D5
:102C3000C4F81C6883BB1D4BA3614FF0FF33636175
:102C4000A36843F00103A36070BD194B9842C9D13A
:102C5000134B4FF08060D3F8D82042F00072C3F8D5
:102C6000D820D3F8002142F00072C3F80021D3F835
:102C70000021D3F8802042F00072C3F88020D3F8FE
:102C8000802022F00072C3F88020D3F88030FFF754
:102C90000FFF0E214D209EE7064BCDE7F4450020A7
:102CA000004402584014004003002002003C30C0A1
:102CB00090460020083C30C0F8B5D0F8904005465A
:102CC00000214FF000662046FFF730FFD5F8941042
:102CD00000234FF001128F684FF0FF30C4F83438F2
:102CE000C4F81C2804EB431201339F42C2F8006968
:102CF000C2F8006BC2F80809C2F8080BF2D20B68E0
:102D0000D5F89020C5F898306362102313611669D6
:102D100016F01006FBD11220FFF772F9D4F8003834
:102D200023F4FE63C4F80038A36943F4402343F05E
:102D30001003A3610923C4F81038C4F814380B4BEE
:102D4000EB604FF0C043C4F8103B094BC4F8003BA4
:102D5000C4F81069C4F80039D5F8983003F11002AE
:102D600043F48013C5F89820A362F8BD8C43000893
:102D700040800010D0F8902090F88A10D2F80038E7
:102D800023F4FE6343EA0113C2F8003870470000E1
:102D90002DE9F84300EB8103D0F890500C468046B3
:102DA000DA680FFA81F94801166806F00306731E07
:102DB000022B05EB41134FF0000194BFB604384ECF
:102DC000C3F8101B4FF0010104F1100398BF06F186
:102DD000805601FA03F3916998BF06F50046002971
:102DE0003AD0578A04F15801374349016F50D5F85A
:102DF0001C180B430021C5F81C382B180127C3F8F9
:102E00001019A7405369611E9BB3138A928B9B08CC
:102E1000012A88BF5343D8F89820981842EA034300
:102E200001F140022146C8F89800284605EB8202CD
:102E30005360FFF77BFE08EB8900C3681B8A43EAF7
:102E4000845348341E4364012E51D5F81C381F4367
:102E5000C5F81C78BDE8F88305EB4917D7F8001BC7
:102E600021F40041C7F8001BD5F81C1821EA030320
:102E7000C0E704F13F030B4A2846214605EB8303D4
:102E80005A60FFF753FE05EB4910D0F8003923F4E0
:102E90000043C0F80039D5F81C3823EA0707D7E704
:102EA0000080001000040002D0F894201268C0F8DE
:102EB0009820FFF70FBE00005831D0F8903049013C
:102EC0005B5813F4004004D013F4001F0CBF022021
:102ED000012070474831D0F8903049015B5813F415
:102EE000004004D013F4001F0CBF022001207047E3
:102EF00000EB8101CB68196A0B6813604B68536063
:102F00007047000000EB810330B5DD68AA691368E3
:102F1000D36019B9402B84BF402313606B8A1468B7
:102F2000D0F890201C4402EB4110013C09B2B4FBE4
:102F3000F3F46343033323F0030343EAC44343F04E
:102F4000C043C0F8103B2B6803F00303012B0ED1E4
:102F5000D2F8083802EB411013F4807FD0F8003B20
:102F600014BF43F0805343F00053C0F8003B02EB22
:102F70004112D2F8003B43F00443C2F8003B30BD9D
:102F80002DE9F041D0F8906005460C4606EB411360
:102F9000D3F8087B3A07C3F8087B08D5D6F814386D
:102FA0001B0704D500EB8103DB685B689847FA07D1
:102FB0001FD5D6F81438DB071BD505EB8403D96879
:102FC000CCB98B69488A5A68B2FBF0F600FB16222E
:102FD0008AB91868DA6890420DD2121AC3E900243F
:102FE000302383F3118821462846FFF78BFF84F3B3
:102FF0001188BDE8F081012303FA04F26B8923EA0A
:1030000002036B81CB68002BF3D021462846BDE834
:10301000F041184700EB81034A0170B5DD68D0F834
:1030200090306C692668E66056BB1A444FF4002065
:10303000C2F810092A6802F00302012A0AB20ED16E
:10304000D3F8080803EB421410F4807FD4F8000989
:1030500014BF40F0805040F00050C4F8000903EB6A
:103060004212D2F8000940F00440C2F800090122DF
:10307000D3F8340802FA01F10143C3F8341870BDE3
:1030800019B9402E84BF4020206020681A442E8A3F
:103090008419013CB4FBF6F440EAC44040F000500F
:1030A000C6E700002DE9F843D0F8906005460C46CD
:1030B0004F0106EB4113D3F8088918F0010FC3F84C
:1030C00008891CD0D6F81038DB0718D500EB81032F
:1030D000D3F80CC0DCF81430D3F800E0DA68964579
:1030E00030D2A2EB0E024FF000091A60C3F8049030
:1030F000302383F31188FFF78DFF89F3118818F0CF
:10310000800F1DD0D6F834380126A640334217D0A0
:1031100005EB84030134D5F89050D3F80CC0E4B229
:103120002F44DCF8142005EB0434D2F800E0516899
:10313000714514D3D5F8343823EA0606C5F8346847
:10314000BDE8F883012303FA01F2038923EA0203AD
:103150000381DCF80830002BD1D09847CFE7AEEBE5
:103160000103BCF81000834228BF0346D7F81809B2
:1031700080B2B3EB800FE3D89068A0F1040959F84E
:10318000048FC4F80080A0EB09089844B8F1040F3C
:10319000F5D818440B4490605360C8E72DE9F84F08
:1031A000D0F8905004466E69AB691E4016F4805802
:1031B0006E6103D0BDE8F84FFEF734BC002E12DA82
:1031C000D5F8003E9B0705D0D5F8003E23F0030359
:1031D000C5F8003ED5F80438204623F00103C5F8B1
:1031E0000438FEF74DFC370505D52046FFF772FC85
:1031F0002046FEF733FCB0040CD5D5F8083813F0A0
:10320000060FEB6823F470530CBF43F4105343F4E0
:10321000A053EB6031071BD56368DB681BB9AB6952
:1032200023F00803AB612378052B0CD1D5F8003EC1
:103230009A0705D0D5F8003E23F00303C5F8003EF9
:103240002046FEF71DFC6368DB680BB120469847FB
:10325000F30200F1BA80B70226D5D4F89090002787
:103260004FF0010A09EB4712D2F8003B03F4402368
:10327000B3F5802F11D1D2F8003B002B0DDA628913
:103280000AFA07F322EA0303638104EB8703DB688E
:10329000DB6813B13946204698470137D4F894309B
:1032A000FFB29B689F42DDD9F00619D5D4F8900093
:1032B000026AC2F30A1702F00F0302F4F012B2F529
:1032C000802F00F0CA80B2F5402F09D104EB8303B0
:1032D000002200F58050DB681B6A974240F0B08006
:1032E0003003D5F8185835D5E90303D50021204619
:1032F000FFF746FEAA0303D501212046FFF740FE53
:103300006B0303D502212046FFF73AFE2F0303D5B6
:1033100003212046FFF734FEE80203D504212046AE
:10332000FFF72EFEA90203D505212046FFF728FE50
:103330006A0203D506212046FFF722FE2B0203D5A1
:1033400007212046FFF71CFEEF0103D50821204688
:10335000FFF716FE700340F1A780E90703D50021AF
:103360002046FFF79FFEAA0703D501212046FFF75D
:1033700099FE6B0703D502212046FFF793FE2F0726
:1033800003D503212046FFF78DFEEE0603D5042169
:103390002046FFF787FEA80603D505212046FFF744
:1033A00081FE690603D506212046FFF77BFE2A062B
:1033B00003D507212046FFF775FEEB0574D520469F
:1033C0000821BDE8F84FFFF76DBED4F890904FF09C
:1033D000000B4FF0010AD4F894305FFA8BF79B682A
:1033E0009F423FF638AF09EB4713D3F8002902F4A8
:1033F0004022B2F5802F20D1D3F80029002A1CDA10
:10340000D3F8002942F09042C3F80029D3F80029EC
:10341000002AFBDB3946D4F89000FFF787FB2289AE
:103420000AFA07F322EA0303238104EB8703DB682C
:103430009B6813B13946204698470BF1010BCAE748
:10344000910701D1D0F80080072A02F101029CBF48
:1034500003F8018B4FEA18283FE704EB830300F5DC
:103460008050DA68D2F818C0DCF80820DCE9001CCB
:10347000A1EB0C0C00218F4208D1DB689B699A6894
:103480003A449A605A683A445A6029E711F0030FA7
:1034900001D1D0F800808C4501F1010184BF02F810
:1034A000018B4FEA1828E6E7BDE8F88F08B5034816
:1034B000FFF774FEBDE8084000F074BBF44500203F
:1034C00008B50348FFF76AFEBDE8084000F06ABB94
:1034D00090460020D0F8903003EB4111D1F8003B2A
:1034E00043F40013C1F8003B70470000D0F890305F
:1034F00003EB4111D1F8003943F40013C1F800394E
:1035000070470000D0F8903003EB4111D1F8003B38
:1035100023F40013C1F8003B70470000D0F890304E
:1035200003EB4111D1F8003923F40013C1F800393D
:1035300070470000090100F16043012203F5614377
:10354000C9B283F8001300F01F039A4043099B009F
:1035500003F1604303F56143C3F880211A607047AB
:1035600030B50433039C0172002104FB0325C160C4
:10357000C0E90653049B0363059BC0E90000C0E952
:103580000422C0E90842C0E90A11436330BD0000CB
:103590000022416AC260C0E90411C0E90A226FF04A
:1035A0000101FEF79DBD0000D0E90432934201D134
:1035B000C2680AB9181D7047002070470369196076
:1035C0000021C2680132C260C26913448269934219
:1035D000036124BF436A0361FEF776BD38B5044634
:1035E0000D46E3683BB162690020131D1268A362B7
:1035F0001344E36207E0237A33B929462046FEF7F5
:1036000053FD0028EDDA38BD6FF00100FBE7000044
:10361000C368C269013BC360436913448269934232
:10362000436124BF436A436100238362036B03B198
:103630001847704770B53023044683F31188866AB3
:103640003EB9FFF7CBFF054618B186F3118828462F
:1036500070BDA36AE26A13F8015B9342A36202D3CE
:103660002046FFF7D5FF002383F31188EFE7000022
:103670002DE9F84F04460E46174698464FF030099C
:1036800089F311880025AA46D4F828B0BBF1000FB1
:1036900009D141462046FFF7A1FF20B18BF31188E5
:1036A0002846BDE8F88FD4E90A12A7EB050B521A99
:1036B000934528BF9346BBF1400F1BD9334601F118
:1036C000400251F8040B914243F8040BF9D1A36A6C
:1036D000403640354033A362D4E90A239A4202D3EC
:1036E0002046FFF795FF8AF31188BD42D8D289F3AF
:1036F0001188C9E730465A46FDF7AEFBA36A5E441F
:103700005D445B44A362E7E710B5029C0433017299
:1037100003FB0421C460C0E906130023C0E90A3397
:10372000039B0363049BC0E90000C0E90422C0E9D5
:103730000842436310BD0000026A6FF00101C260DD
:10374000426AC0E904220022C0E90A22FEF7C8BC8E
:10375000D0E904239A4201D1C26822B9184650F830
:10376000043B0B60704700231846FAE7C36800214A
:10377000C2690133C3604369134482699342436160
:1037800024BF436A4361FEF79FBC000038B504467E
:103790000D46E3683BB1236900201A1DA262E2696D
:1037A0001344E36207E0237A33B929462046FEF743
:1037B0007BFC0028EDDA38BD6FF00100FBE700006C
:1037C00003691960C268013AC260C2691344826920
:1037D0009342036124BF436A036100238362036B46
:1037E00003B118477047000070B530230D460446FA
:1037F000114683F31188866A2EB9FFF7C7FF10B10F
:1038000086F3118870BDA36A1D70A36AE26A013352
:103810009342A36204D3E16920460439FFF7D0FF45
:10382000002080F31188EDE72DE9F84F04460D469E
:10383000904699464FF0300A8AF311880026B34625
:10384000A76A4FB949462046FFF7A0FF20B187F38A
:1038500011883046BDE8F88FD4E90A073A1AA8EB78
:103860000607974228BF1746402F1BD905F1400392
:1038700055F8042B9D4240F8042BF9D1A36A403639
:103880004033A362D4E90A239A4204D3E169204673
:103890000439FFF795FF8BF311884645D9D28AF397
:1038A0001188CDE729463A46FDF7D6FAA36A3D448A
:1038B0003E443B44A362E5E7D0E904239A4217D192
:1038C000C3689BB1836A8BB1043B9B1A0ED0136013
:1038D000C368013BC360C3691A4483699A420261A9
:1038E00024BF436A036100238362012318467047A3
:1038F0000023FBE700F080B94FF08043586A70471F
:103900004FF08043002258631A610222DA60704748
:103910004FF080430022DA60704700004FF0804390
:1039200058637047FEE7000070B51B4B0025044646
:1039300086B058600E468562016300F00BF904F111
:103940001003A560E562C4E904334FF0FF33C4E916
:103950000044C4E90635FFF7CFFF2B46024604F1C9
:1039600034012046C4E9082380230C4A2565FEF76C
:1039700051FB01230A4AE0600092037568467268B1
:103980000192B268CDE90223064BCDE90435FEF77A
:1039900069FB06B070BD00BFB02A0020C843000814
:1039A000CD43000825390008024AD36A1843D06283
:1039B000704700BF482800204B6843608B688360D5
:1039C000CB68C3600B6943614B6903628B694362D7
:1039D0000B6803607047000008B53C4B40F2FF7174
:1039E0003B48D3F888200A43C3F88820D3F88820BE
:1039F00022F4FF6222F00702C3F88820D3F888205F
:103A0000D3F8E0200A43C3F8E020D3F808210A43A2
:103A1000C3F808212F4AD3F808311146FFF7CCFF2D
:103A200000F5806002F11C01FFF7C6FF00F5806021
:103A300002F13801FFF7C0FF00F5806002F1540188
:103A4000FFF7BAFF00F5806002F17001FFF7B4FFE5
:103A500000F5806002F18C01FFF7AEFF00F5806099
:103A600002F1A801FFF7A8FF00F5806002F1C40190
:103A7000FFF7A2FF00F5806002F1E001FFF79CFF75
:103A800000F5806002F1FC01FFF796FF02F58C71F2
:103A900000F58060FFF790FF00F074F90E4BD3F84B
:103AA000902242F00102C3F89022D3F8942242F00F
:103AB0000102C3F894220522C3F898204FF0605207
:103AC000C3F89C20054AC3F8A02008BD0044025852
:103AD00000000258D443000800ED00E01F00080376
:103AE00008B500F031FBFEF759FA0F4BD3F8DC2094
:103AF00042F04002C3F8DC20D3F8042122F0400257
:103B0000C3F80421D3F80431084B1A6842F00802C4
:103B10001A601A6842F004021A60FEF727FFBDE837
:103B20000840FEF7C9BC00BF004402580018024814
:103B300070470000EFF30983054968334A6B22F0B0
:103B400001024A6383F30988002383F311887047D5
:103B500000EF00E0302080F3118862B60D4B0E4A72
:103B6000D96821F4E0610904090C0A430B49DA60C1
:103B7000D3F8FC2042F08072C3F8FC20084AC2F857
:103B8000B01F116841F0010111602022DA7783F83B
:103B90002200704700ED00E00003FA0555CEACC5E9
:103BA000001000E0302310B583F311880E4B5B68E2
:103BB00013F4006314D0F1EE103AEFF309844FF0E0
:103BC0008073683CE361094BDB6B236684F30988EF
:103BD000FEF7B8F910B1064BA36110BD054BFBE72A
:103BE00083F31188F9E700BF00ED00E000EF00E08B
:103BF0002F04000832040008114BD3F8E82042F0EB
:103C00000102C3F8E820D3F8102142F00102C3F802
:103C100010210C4AD3F81031D36B43F00103D36366
:103C20004FF08043C7229A624FF0FF32DA620022DF
:103C30009A615A63DA605A6001225A611A607047C9
:103C4000004402580010005C4FF0804208B5116932
:103C5000D3680B40D9B29B076FEA0101116107D508
:103C6000302383F31188FEF7AFF9002383F3118823
:103C700008BD0000064BD3F8DC200243C3F8DC206B
:103C8000D3F804211043C3F80401D3F8043170477A
:103C9000004402583A4B4FF0FF31D3F8802062F0D5
:103CA0000042C3F88020D3F8802002F00042C3F81D
:103CB0008020D3F88020D3F88420C3F88410D3F870
:103CC00084200022C3F88420D3F88400D86F40F009
:103CD000FF4040F4FF0040F4DF4040F07F00D86731
:103CE000D86F20F0FF4020F4FF0020F4DF4020F0E8
:103CF0007F00D867D86FD3F888006FEA40506FEA2A
:103D00005050C3F88800D3F88800C0F30A00C3F805
:103D10008800D3F88800D3F89000C3F89010D3F847
:103D20009000C3F89020D3F89000D3F89400C3F823
:103D30009410D3F89400C3F89420D3F89400D3F8E7
:103D40009800C3F89810D3F89800C3F89820D3F8D7
:103D50009800D3F88C00C3F88C10D3F88C00C3F80B
:103D60008C20D3F88C00D3F89C00C3F89C10D3F8B7
:103D70009C10C3F89C20D3F89C3000F0B9B900BF68
:103D80000044025808B50122534BC3F80821534B95
:103D9000D3F8F42042F00202C3F8F420D3F81C2137
:103DA00042F00202C3F81C210222D3F81C314C4B12
:103DB000DA605A689104FCD54A4A1A6001229A6076
:103DC000494ADA6000221A614FF440429A61444B3A
:103DD0009A699204FCD51A6842F480721A603F4BCB
:103DE0001A6F12F4407F04D04FF480321A67002219
:103DF0001A671A6842F001021A60384B1A685007B5
:103E0000FCD500221A611A6912F03802FBD1012197
:103E100019604FF0804159605A67344ADA62344A77
:103E20001A611A6842F480321A602C4B1A689103A6
:103E3000FCD51A6842F480521A601A689204FCD5C4
:103E40002C4A2D499A6200225A63196301F57C01BC
:103E5000DA6301F2E71199635A64284A1A64284A1E
:103E6000DA621A6842F0A8521A601C4B1A6802F013
:103E70002852B2F1285FF9D148229A614FF4886242
:103E8000DA6140221A621F4ADA641F4A1A651F4A21
:103E90005A651F4A9A6532231E4A1360136803F05D
:103EA0000F03022BFAD10D4A136943F00303136188
:103EB000136903F03803182BFAD14FF00050FFF7C5
:103EC000D9FE4FF08040FFF7D5FE4FF00040BDE82F
:103ED0000840FFF7CFBE00BF0080005100440258E9
:103EE0000048025800C000F0020000010000FF017D
:103EF000008890081210200063020901470E05088F
:103F0000DD0BBF0120000020000001100910E000BF
:103F100000010110002000524FF0B04208B5D2F865
:103F2000883003F00103C2F8883023B1044A1368D3
:103F30000BB150689847BDE80840FFF733BE00BF9B
:103F4000444700204FF0B04208B5D2F8883003F063
:103F50000203C2F8883023B1044A93680BB1D068D9
:103F60009847BDE80840FFF71DBE00BF444700204A
:103F70004FF0B04208B5D2F8883003F00403C2F81D
:103F8000883023B1044A13690BB150699847BDE8E2
:103F90000840FFF707BE00BF444700204FF0B04283
:103FA00008B5D2F8883003F00803C2F8883023B18E
:103FB000044A93690BB1D0699847BDE80840FFF700
:103FC000F1BD00BF444700204FF0B04208B5D2F821
:103FD000883003F01003C2F8883023B1044A136A12
:103FE0000BB1506A9847BDE80840FFF7DBBD00BF42
:103FF000444700204FF0B04310B5D3F8884004F494
:104000007872C3F88820A30604D5124A936A0BB1CC
:10401000D06A9847600604D50E4A136B0BB1506BFB
:104020009847210604D50B4A936B0BB1D06B984788
:10403000E20504D5074A136C0BB1506C9847A305F1
:1040400004D5044A936C0BB1D06C9847BDE810407E
:10405000FFF7A8BD444700204FF0B04310B5D3F898
:10406000884004F47C42C3F88820620504D5164ACF
:10407000136D0BB1506D9847230504D5124A936D0B
:104080000BB1D06D9847E00404D50F4A136E0BB105
:10409000506E9847A10404D50B4A936E0BB1D06EB5
:1040A0009847620404D5084A136F0BB1506F9847C4
:1040B000230404D5044A936F0BB1D06F9847BDE831
:1040C0001040FFF76FBD00BF4447002008B503480C
:1040D000FDF744F8BDE80840FFF764BDD823002091
:1040E00008B5FFF7B1FDBDE80840FFF75BBD000074
:1040F000062108B50846FFF71DFA06210720FFF73D
:1041000019FA06210820FFF715FA06210920FFF702
:1041100011FA06210A20FFF70DFA06211720FFF7F2
:1041200009FA06212820FFF705FA09217A20FFF76E
:1041300001FA07211C20FFF7FDF90C213520BDE80D
:104140000840FFF7F7B9000008B5FFF7A3FD00F03E
:104150000DF8FDF71BFAFDF7F3FBFDF7C5FAFFF7C6
:10416000E7FCBDE80840FFF7C5BB00000023054A97
:1041700019460133102BC2E9001102F10802F8D1EF
:10418000704700BF4447002010B5013902449042F7
:1041900001D1002005E0037811F8014FA34201D0BE
:1041A000181B10BD0130F2E7034611F8012B03F88C
:1041B000012B002AF9D1704753544D333248373F11
:1041C0003F3F0053544D3332483733782F373278DE
:1041D0000053544D3332483734332F3735332F376C
:1041E0003530000001105A0003105900012058001A
:1041F00003205600009600000000000000000000B0
:1042000000000000000000000000000000000000AE
:104210004D150008391500087515000861150008CE
:104220006D150008591500084515000831150008DE
:1042300081150008000000006516000851160008EE
:104240008D160008791600088516000871160008FA
:104250005D160008491600089916000800000000C5
:104260000100000000000000633000006842000808
:10427000A0280020B02A00204172647550696C6F3C
:10428000740025424F415244252D424C0025534590
:104290005249414C250000000200000000000000CF
:1042A00085180008F5180008400040006043002011
:1042B0007043002002000000000000000300000026
:1042C000000000003D190008000000001000000080
:1042D00080430020000000000100000000000000FA
:1042E000F445002001010200552400086523000860
:1042F00001240008E52300084300000000430008F3
:1043000009024300020100C0320904000001020258
:10431000010005240010010524010001042402020B
:104320000524060001070582030800FF09040100B7
:10433000020A000000070501024000000705810293
:1043400040000000120000004C4300081201100160
:10435000020000400912415700020102030100005F
:104360000403090425424F4152442500466C7969F3
:104370006E674D6F6F6E48373433003031323334EF
:104380003536373839414243444546000000000085
:10439000991A0008511D0008FD1D0008400040004A
:1043A0002C4700202C470020010000003C47002043
:1043B0008000000040010000080000000001000033
:1043C00000100000080000006D61696E0069646CF7
:1043D000650000000001912A00000000AAAA8AAA34
:1043E00000011124FFFF00000000000000A00A00EF
:1043F0001500000000000000AAAAAAAA15000000EB
:10440000FFFF0000000000000000000000000002AC
:1044100000000000AAAAAAAA00000001FFFF0000F5
:104420000000000000000800200000000000000064
:10443000AAAAAAAA10000000FFFF000000080000BE
:10444000000000005000004000000000AAAAAAAA34
:1044500000000040FFFF000000000000000000001E
:104460000000000000000000AAAAAAAA00000000A4
:10447000FFFF00000000000000000000000000003E
:1044800000000000AAAAAAAA00000000FFFF000086
:10449000000000000000000000000000000000001C
:1044A000AAAAAAAA00000000FFFF00000000000066
:1044B000000000000000000000000000AAAAAAAA54
:1044C00000000000FFFF00000000000000000000EE
:1044D0000000000000000000AAAAAAAA0000000034
:1044E000FFFF0000000000000000000000000000CE
:1044F00000000000AAAAAAAA00000000FFFF000016
:10450000000000000000000058040000000000004F
:1045100000001E0000000000FF000000B82A00207C
:10452000D823002000000000B841000883040000E8
:10453000C341000850040000D1410008009600006B
:1045400000000800960000000008000004000000C1
:1045500060430008000000000000000000000000B0
:0C4560000000000000000000000000004F
:00000001FF
